:020000040000FA
:060000000219FD02031CC1
:03000B0002008D63
:03001300020537AC
:03001B0002009050
:03002B000202D1FD
:03005B0002054655
:030073000203097C
:100080000406080C10182030406080A0C0054032E3
:10009000C2AFC2A853E6EFC28E856B8BC0D0D2D35D
:1000A000C0E0C0F0C2CAA8CCA9CDD2CAD2AF758A6E
:1000B00000C3E8956CF8E9956DF9C3E913F9E81305
:1000C000F8E5666007C3E913F9E813F8E97025E875
:1000D000956E4020956E501CE582B410177C007B15
:1000E000007A007908900000A86AE5667004C3E809
:1000F00013F801FD900000D2A8D2AA61E7E0FDC389
:100100009CC39840EF98EB33FB0582E0FCC39DC392
:100110009840E198EB33FB0582E0FDC39CC3984017
:10012000D398EB33FB0582E0FCC39DC39840C59890
:10013000EB33FB0582E0FDC39CC39840B798EB33DB
:10014000FB0582E0FCC39DC39840A998EB33FB05F7
:1001500082E0FDC39CC398409B98EB33FB0582E093
:10016000FCC39DC398408D98EB33FB0582217890AA
:100170000000D2A8D2AA61E7E0FDC39CC39840EF7B
:1001800098EA33FA0582E0FCC39DC39840E198EAFF
:1001900033FA0582E0FDC39CC39840D398EA33FA52
:1001A0000582E0FCC39DC39840C598EA33FA0582F6
:1001B000E0FDC39CC39840B798EA33FA0582E0FC9F
:1001C000C39DC39840A998EA33FA0582E0FDC39C19
:1001D000C398409B98EA33FA0582E0FCC39DC3981C
:1001E000408D98EA33FA0582EBC46B6A54F0F9EA61
:1001F000C454F0C3996009900000D2A8D2AA61E764
:10020000EBF4C454F0F9EAF4C4540F49FAEBF4C423
:10021000540FFBC3EAF99460FAEB9400FB5020C33F
:10022000E97B007A0079006016C3135006F9C39584
:1002300052600AE9F5527553007900800205533087
:100240003A27C3EA94D0F8EB9407F9400BE8FAE9AF
:10025000FB203509D235415D303502C235203902E7
:10026000B235C3EA33FAEB33FBEB2B3B3BF9C3EB81
:1002700013FBEA13FAEA29FAEB3400FB30E3047AC1
:10028000FF7BFFE5255403601B202A18E55D33F949
:10029000EB7007C3E99A4002E9FAE53CC4332AFA55
:1002A000EB3400FBC3EA33C4540FF8EB33C454F00F
:1002B00048F87005EA60027801900000D2A8D2AA3E
:1002C000E5226002152281D4900000D2A8D2AA6152
:1002D000E7C0D0C0E0C2CF0541E5666009E56560D2
:1002E000057565006104756501E52360021523C38A
:1002F000E55460057555006104E5552401F5555038
:10030000037555FFD0E0D0D032C2AF53E67F75926F
:10031000FA7593FFC22053917FD2AF32C0E0E58AD5
:10032000303408856B8BF0A3D0E032D0E0C2AF53FD
:10033000E6EFC0D0C0E0C0F0D2D3D2AF5388EFA870
:100340008AA98CAA40308D010A758A00758C0075C7
:100350004000438810E566700AC3E833F8E933F9D2
:10036000EA33FA30331FE8C4540FFAE9C454F04AB0
:10037000FAC3132AFAC3E833F8E933F9E82AFAE9A9
:100380003406FB61D830320FC3E833E933FAE82A88
:10039000FAE93400FB61D8303115E875F056A4AAAB
:1003A000F0E975F056A42AFAC5F03400FB61D8C311
:1003B000EA13FAE913F9E813F8E875F056A4AAF07D
:1003C000E975F056A42AFAC5F03400C313FBEA130A
:1003D000FAC3EB13FBEA13FAC3EB94125009C3EA16
:1003E0009434EB940750160522E52270021522C3BF
:1003F000E52294325002A12A755400A12DE5226015
:100400000215223036067C007D088117AC31AD32F2
:10041000303A04AC33AD34C3EA9CFAEB9DFB92084E
:10042000AE60AF61303A425007203509D235813590
:10043000303502C235303504AE62AF63203902B2C6
:1004400035C3EA33FAEB33FBA208500AEAF424017D
:10045000FAEBF43400FBC3EA9450FAEB9400FB503F
:100460001478007A007B008175A208500878007A21
:10047000007B0081D4E5255403601B202A18E55D2C
:1004800033F9EB7007C3E99A4002E9FAE53CC4335B
:100490002AFAEB3400FBEA8EF0A4F9AAF0EB8EF016
:1004A000A42AFAC5F03400FBC3EB13FDEA13F8C32A
:1004B000ED13FDE813F80FEF146004C3E833F8C33D
:1004C000E933EA33FAEB33FBDFEDEB30E30678FF99
:1004D0007AFF7B078854D230E86003755500C3E586
:1004E0005BFC955C4002AC5CC3EC95545008EC7529
:1004F000F008A4FAABF0EAF4F8EBF45407F98856E4
:10050000895775230AE55A30E210D0F0D0E0D0D0F8
:1005100053F7DF43F74043E61032D0F0D0E0D0D0BD
:1005200053D8FE43DA0143E6103275230AD0F0D0E7
:10053000E0D0D043E61032C2AAD28EC2CA85CC6CBB
:1005400085CD6DD2CA32C2AFC0D0C0E0D2D38556FD
:10055000FB8557FC85575A53F7BF53DAFED2A830B4
:100560003402D2AA53E6EF53F7DF53D8FED0E0D0DF
:10057000D0D2AF327901801479038010790A800CCF
:10058000791E80087964800479C880007817E4D5E2
:10059000E0FDD8FAD9F62278FF20282879A1E76073
:1005A00023E548601F74FF8548F084853FF03029BB
:1005B0000375F005A4F8C5F0600278FFC3E8955D07
:1005C0005002A85D885C22C3E54794A0E5489400EA
:1005D000E55C500314A1D8046002F55C2275E89034
:1005E00022055EC3E55E9408405330EDF4A8BDA932
:1005F000BE755E00E9FA79A0E76041EA7006E55F42
:100600006018800CC3E8955F600EE55F5005600AD6
:100610001480070460FA8002E55FF55FC3956940C6
:100620001B755BC0C394044013755B80C394044086
:100630000B755B40C394044003755B0022E55B24AB
:1006400010500274FFF55B22743279A687F0A4C5BE
:10065000F0A2F733F55D227547007548F022C2AF6E
:10066000C2CAA8CCA9CDAA4130CF010AD2CAD2AF02
:10067000C3EA13FAE913F9E813F8AB42AC43884232
:100680008943C3E89BF8E99C20280A547FF9302C61
:1006900002E17CC1D5AD448A44F9EA9D547FFA60F9
:1006A0000678FF79FFC1BAAE45AF468B458C46A8A8
:1006B00042A943C3E89EF8E99FF9C3E54813FBE567
:1006C0004713FAE82AF547E93BF54850067547FF16
:1006D0007548FFE122AA47AB48AC47AD487E047F8E
:1006E00002C3EB9404400D1E1FC3EB940840052089
:1006F00029021E1FC3ED13FDEC13FCDEF7C3EA9CB9
:10070000FAEB9DFBEF6009C3E913F9E813F8DFF793
:10071000EA28FAEB39FB8A478B4850067BFF8B4768
:100720008B48C3EB94025002D22C3028047F03E1A3
:100730004D7892E6FFC3E53D948240110FC3E53D3D
:1007400094A040010FC3EF940640027F057E02E5AE
:1007500048C4540FF9E548C454F0F8E547C4540FB1
:1007600028F8C3E89EFAE99400FB4009C3EA940123
:10077000EB940050047A01E4FB0207C8AA47AB4897
:10078000EBC4FEEAC4540F4EFCC3EA9CFAEB94009F
:10079000FBC3E813C313F8EA28FAEB3400FB8A47DB
:1007A0008B48C3EB94024002C22C7802EBC4FE7B60
:1007B00000EAC4540F4EFAC3EA98FA4005C3940104
:1007C00050027A017892E6FF302002E1C8854E920D
:1007D000854F93D22043E680C3E49AF8E49BF9C3A3
:1007E000E833F8E933F9302C0302085DE8FAE9FB55
:1007F000D3E913FDE813FC884E894FC3EF940360DF
:1008000038EF20E00CE82CF8E93DF9ECFAEDFB803C
:1008100013E828F8E939F9C3E82401F8E93400F9C4
:100820007AFF7BFFC3EF9403400F8A508B51884AB5
:10083000894B8C4C8D4D020892885089518A4A8B85
:100840004B8C4C8D4D3028127550F07551FF754C06
:10085000F0754DFF754EF0754FFF020892E8FAD320
:10086000E813FC884EC3EF94036021EF20E007E813
:100870002CF8ECFA017DE8282401F87AFFC3EF9404
:100880000340098A50884A8C4C02089288508A4A50
:100890008C4C3020020192753A02D22043E680E56A
:1008A000255403602DA847A948C3E913F9E813F8B4
:1008B000302804E92440F9C2AF53E67F759100C3A4
:1008C000E498F594E499F595759104D22043E68077
:1008D000D2AF22D221754900752000302B0375203C
:1008E0004001F1D221754900752040302B0375205D
:1008F0000078017901202C20E52554036002C221F3
:100900007914E548C313700104F8C39414400278C5
:1009100014302804781B791BC3E833F8C3E933F992
:10092000202010E549600C302803D53A04D222215A
:10093000A4119A0549E59B5440B52002218E302828
:100940000908C3E899400118212020210A08C3E8BA
:1009500099400201F12120C22153E67F75910030B8
:100960002C117594007595F0759104D22043E680A2
:100970000208F1E5487EFFC3334009C3334005C395
:10098000334001FEC3E49E759400F5952168C3E5EC
:10099000399401500201F130210201F1D80221A263
:1009A0002120C222C2AF53E67F7591008550948505
:1009B0005195759104854A92854B93D22043E680E8
:1009C000D2AFE52554036007202902053980103095
:1009D000220D202B0A2021071581158102140B22DC
:1009E00078003021027801E53D75F007A4F9E5F0C3
:1009F00028F5F0E9A2F013A2F113A2F213F53DC31A
:100A000094785003753D78C3E53D953E400653F21A
:100A10008F75D5FF3020024114854C92854D93D2BD
:100A20002043E68022203817C2AF53F2DFC296433C
:100A3000F24075D5EF43F210D2AF759F536149C2B2
:100A4000AF53F2DFC29443F21075D5BF43F240D2E8
:100A5000AF759F536149203817C2AF53F2EF75D578
:100A6000DF43F220C29643F240D2AF759F636149E3
:100A7000C2AF53F2BF75D5DF43F220C29443F210E8
:100A8000D2AF759F236149203817C2AF53F2BFC25E
:100A90009443F21075D5DF43F220D2AF759F2361E6
:100AA00049C2AF53F2EFC29643F24075D5DF43F22D
:100AB00020D2AF759F636149203817C2AF53F2DF70
:100AC00075D5BF43F240C29443F210D2AF759F5325
:100AD0008077C2AF53F2DF75D5EF43F210C2964371
:100AE000F240D2AF759F538060203817C2AF53F2E7
:100AF000EFC29543F22075D5BF43F240D2AF759F48
:100B0000638046C2AF53F2BFC29543F22075D5EF62
:100B100043F210D2AF759F23802F203817C2AF53F6
:100B2000F2BF75D5EF43F210C29543F220D2AF75F4
:100B30009F238015C2AF53F2EF75D5BF43F240C279
:100B40009543F220D2AF759F63227A147B7880128E
:100B50007A107B8C800C7A0D7BB480067A0B7BC874
:100B60008000E564D5E001227902E453F2DFD5E0AC
:100B7000FDD29543F220D5E0FD53F2DFD5E0FDC272
:100B80009543F220D5E0FDE920E005D29643F240FE
:100B900030E005D29443F210E564D5E0FDE920E0B1
:100BA0000353F2BF30E00353F2EF7496D5E0FDD962
:100BB000B9EAF8D5E0FDD8FBDBA853F2DF2253F207
:100BC0008F53F28F75D5FF22788076FF0876FF0865
:100BD00076FF0876FF0876FF0876FF087609087624
:100BE000FF087601788C76010876FF0876FF087694
:100BF000FF0876FF0876FF0876030876FF0876FF81
:100C00000876FF0876250876D008762808765008FA
:100C100076040876FF0876020876FF08767A08766A
:100C2000FF0876070876010876FF0876FF08760049
:100C300008760022FA75F00CA4ABF0EAC333F8741E
:100C40000133F9E8C333F8E933F9E8C32BF8E934A1
:100C500000F9E8C333F8E933F9227888E6C394034E
:100C6000D23A5002C23AC238E630E102D238A23853
:100C700092397886E6149000809378A6F67886E616
:100C8000F53FC394025003753F02789CE6753EFF22
:100C9000B40203753EA0B40303753E8278A0E6F863
:100CA000600674282409D8FCF5697896E6913488A2
:100CB000318932789EE69134883389347897E69189
:100CC000348835893671BE223036117A007B007C3B
:100CD000FF7D007E00B12E8B618A6022303A22783F
:100CE00096E6FA7B00789EE6FC7D00C3EA33FAEBD9
:100CF00033FBC3EC33FCED33FD7E0AB12E8B638AEC
:100D0000627896303A02789EE6FA7B007897E6FCA5
:100D10007D007E00303A10C3EA33FAEB33FBC3ECBC
:100D200033FCED33FD7E0AB12E8B618A6022C3EC69
:100D30009EFCED9400FDC3EC9AFCED9BFDC3EC948E
:100D400023ED940050047C237D00C3EC94FFED94CC
:100D50000140047CFF7D017BFF0B7A000AEA7009E9
:100D6000C3EC33FCED33FDA159EC8AF0A4AEF0EDF9
:100D70008AF0A42E947C40E4EAF460DD22D236911D
:100D8000C81205801205807A007B007C101205785D
:100D9000E5542AFA74003BFBDCF37C04C3EB13FB41
:100DA000EA13FADCF7FFEB60027FFFC23691C8223C
:100DB00078A5E6F954037000E9540C7000E954304A
:100DC0007000E954C070002275670075680075975F
:100DD000DE7597AD7581C043FF8075EF0675A9007C
:100DE00071BE7580FF75F19375A4007580FF75D491
:100DF000FF75900075F28F75A57075900075D5FF21
:100E000075A60175E34075E20271BEE4F8F6D8FDFF
:100E100071C812145878988664753001C2AF1205F3
:100E200088714A1205807150120580715612058032
:100E3000B1B0C2AF75670075680078FA79FA30878B
:100E400007D9FBD8F7021C00915A91C8789886649C
:100E500071BE75A91375A71075C10075A7007566D9
:100E60000075E407758811758E0475890975C804C5
:100E700075910475D84075D90875F783759E00750E
:100E8000960075DA4A75DB0075A82375E69075B88B
:100E900001759B80759D0075D10C75BCB975BB1033
:100EA00075E88075B201120574D2AF753C00C2308E
:100EB000120588C231C232C233C234755200755332
:100EC00000752200120584C3E522940A5002E198BD
:100ED000D231752200120584C3E522940A5002E142
:100EE00098C231D232752200120584C3E522940AD9
:100EF0005002E19875E4F7758851758E017589AADD
:100F0000758C00758D00C2A9D2ABD2AA756B8075A5
:100F10006A14756E50C232D23475220A1205847575
:100F20006A10C3E522940A75520075530040697532
:100F30008E0C756B00756A28756E2875220A12056D
:100F400084756A20C3E522940A75520075530040E7
:100F500047758E0C756B80756A14756E1475220A50
:100F6000120584756A10C3E522940A755200755300
:100F700000402575E407758811758E04758909D2BE
:100F8000A9C2ABC2AAC234D233752200120584C3EF
:100F9000E522940A4002C132120578203003020E85
:100FA00032C2AF714A714A714AD2AF1205882034F9
:100FB00003303A0302105B120578788CE6C3940183
:100FC000500302105BE530C39401500302105B75BF
:100FD00067A57568F17F02D23691C8120584C2AF49
:100FE000C23691C8C3E554947FD2AF406E120574E7
:100FF000C2AF715CD2AFDFDFB17DC3EF7897F6127D
:101000000588B1457F0AD236120CC8120584C2AFDA
:10101000C236120CC8C3E554947FD2AF50E6120515
:1010200074C2AF120B4A12057C120B4AD2AFDFD644
:10103000120D7DEF24037896F6F87997E7C3942391
:101040004003985006E824237897F6120588919F6C
:10105000B174120584120CC8020E327567007568EF
:1010600000120584C3E55494014003020FAEC2AFE1
:10107000120B5C120B5C120B5CD2AF120588753040
:1010800000E4F537F5380537E537F4703F05387873
:101090009AE67819146012783214600D787D146025
:1010A0000878FA146003753800C3E53898401D12BB
:1010B0000BBE120574153875370078998664C2AF77
:1010C000120B5CD2AF7898866412058412057CE519
:1010D000237003020E32C3E5549401500AC3E55253
:1010E00094015016021086120584E5237003020E47
:1010F0003275520075530002129CC3E55294017080
:1011000017C2AF120BBE78998664120B4A78988684
:1011100064D2AF120584418EC3E55294027017C2A7
:10112000AF120BBE78998664120B5078988664D201
:10113000AF120584418EC3E55294037017C2AF12FB
:101140000BBE78998664120B5678988664D2AF12DB
:101150000584418EC3E55294047017C2AF120BBED2
:1011600078998664120B5C78988664D2AF120584F5
:10117000418EC3E55294057017C2AF120BBE789929
:101180008664120B5C78988664D2AF120584418E17
:10119000C3E55294077019C3E5539406500201D673
:1011A0007401303A0274037888F6C238C239418E2D
:1011B000C3E55294087019C3E5539406500201D652
:1011C0007402303A0274047888F6D238D239418EEB
:1011D000C3E55294097017C3E5539406500201D633
:1011E000303A0BC37888E69402F6C23A418EC3E5E2
:1011F00052940A7016C3E5539406500201D6203A61
:101200000A7888E62402F6D23A418EC3E552941455
:101210007025C3E5539406500201D6C2AF901A0B55
:10122000740093D2AF7888F613C238C2394002D224
:10123000384002D2398057C3E55294157038C3E55F
:10124000539406404FC2AF901A0B740093D2AFF87C
:10125000B801027402B802027401B803027404B83F
:10126000040274037888F613C238C2394002D238B7
:101270004002D2398018C3E552940C70117567A5ED
:101280007568F1C3E5539406400A919FD2AF755239
:101290000075530075670075680001D6C2AF120B68
:1012A000BEE4D2AFE4F55EF524F525F53D755E08A4
:1012B0001205741205DD30EDFDA8BDA9BEE970016F
:1012C000F8885F1205E1755E08C2AF120648855DB9
:1012D0005B855D5CD2AF75A71075C13075A70075D1
:1012E000A903756601303A07C238303502D238D2C8
:1012F00028753900120AE9120B1A12065712065EF7
:1013000012065712065E1206571208E31209E0127F
:101310000A2512065E1208D3202C03120597302CE2
:10132000031205C71209E0120A5612065E1208E3FC
:101330001209E0120A8712065E1208D31209E0129F
:101340000AB812065E1208E31209E0120AE9120650
:101350005E1205DD1208D31209E0120B1A1205E124
:1013600012065E302827855D5B79187A0CC3E53953
:1013700099400EC228D2298A3B855D5B855D5C80E1
:101380000CC3E55494014003021309811330291F53
:10139000202B1CE53B147006C229D22A6109F53BBB
:1013A000203A07C3E5549401400302130980647591
:1013B0003C00203A0F78FA79A4E760027803C3E58D
:1013C0005598504FE523604B303A172038052035AB
:1013D00007800F303502800A202B07D22B855D5BFA
:1013E000613978F0302B05855D5B7820C3E548983E
:1013F0005003021309302B1BC22BC238303502D2E6
:1014000038D229753B12855D5B6109053CE5546066
:10141000028116753C00C2AF120BBE752400752503
:101420000075A91375A71075C10075A70075660032
:10143000D2AF120584120BBE78A4E6600FC29643A9
:10144000F240C29543F220C29443F210C3E53C94AB
:10145000044003020E320181901A0D782091D8E5E4
:1014600020B4550AA391D8E520B4AA028013756769
:10147000A57568F1120BC8919F75670075680080AB
:101480001D901A0378807B0A91D8A308DBFA901A82
:101490000F788C7B1A91D8A308DBFA901A2922C204
:1014A000AFB11B91F8901A00741091DDA3740791ED
:1014B000DDA3742191DD901A0378807B0A91DCA36F
:1014C00008DBFA901A0F788C7B1A91DCA308DBFA00
:1014D000B12EB10C901A2922E493F622E6438F0133
:1014E000538FFDFFC3E583941C400122EF8567B74E
:1014F0008568B7F0538FFE22438F02438F018567C3
:10150000B78568B7901A0DF0538FFC22901A0D74AE
:101510005591DD901A0E74AA91DD227A3079D07837
:1015200020901A4091D8E520F709A3DAF7227A3003
:1015300079D0901A40E791DD09A3DAF9227C0512EF
:101540000588DCFB22C2AF120B4A120B50120B565D
:10155000120B5C12057C120B4A120B50120B561226
:101560000B5C12057C120B4A120B50120B56120B1D
:101570005CD2AF22C2AF120B5C120B56120B501290
:101580000B4A12057C120B5C120B56120B50120BFD
:101590004A12057C120B5C120B56120B50120B4AAE
:0315A000D2AF22A5
:1019FD00020DC8100721FFFFFFFFFFFF09FF01FFC9
:101A0D0055AA01FFFFFFFFFF03FFFFFF25D0285061
:0D1A1D0004FF02FF7AFF0701FFFF0000FF3A
:101A400023575F485F303023202020202020202093
:101A500023424C48454C492445464D3842323123B7
:101A60002020202020202020202020202020202076
:101C0000C2AFC2D37597DE7597AD7581C075A90057
:101C100043FF80752438752503B1DB7529A5752A26
:101C2000F143F18053A47FD28775D4FF75E3407DE3
:101C3000FA780379E67C10752200752300901DE880
:101C40007B06752498752501308702814820870816
:101C5000D8FBD9F9DCF781BA308708D8FBD9F9DC91
:101C6000F781BAB19BE493A3C39A6004DDC381BA40
:101C7000DBDBB18D600281317B08E493FAA3B16EA6
:101C8000DBF87A30B16E752200752300B18DEAFC65
:101C9000EBFDC3ED94FE400EB18D8A278B28ED300D
:101CA000E0048A828B83B18D7AC270D8C3ED94FE32
:101CB000601950CEBD0029EC600F7520007521FF22
:101CC000752900752A000200008100A827A92808AC
:101CD00009D804D90281DDB191EAF281D10D81A642
:101CE000C3ED94035051EDA2E092007AC5C3E582A2
:101CF0009400E583941C508C200010438F02438F86
:101D0000018529B7852AB7F0300027A827A9280818
:101D100009438F01538FFDD804D902A132C3E58353
:101D2000941C4003A3A117E28529B7852AB7F0A325
:101D3000A117538FFC81827AC1BD030CE493A3FAEF
:101D4000B152DCF8B14A81828184AA22AB23B16E00
:101D5000EBFAEA6222752608C3E52313F523E52290
:101D600013F52250066323A0632201D526EAB1DBD6
:101D7000B1DB75260AEAF4200102D287300102C2E3
:101D800087B1DBC3134002C201D526EB22B191EA31
:101D9000FB208702A191308702A196752608AE2408
:101DA000AF25C3EF13FFEE13FEB1DFB1DBC3EA13C0
:101DB0003087024480FA30E703632201C3E523132E
:101DC000F523E52213F52250066323A0632201D5F3
:101DD00026D9E52265236523F52222AE24AF250E00
:101DE0000FDEFEDFFCD20122424C48656C693437BD
:061DF0003164E8B20601B7
:00000001FF
